:2000000002014112005C3200000000021B9C000000000032000000000000003200000000DF
:20002000000000C0D0C0E0C0F0C082C083D2D310982510990BD083D082D0F0D0E0D0D0324E
:20004000106F08ECB50B04C26880EAA80C86990CBC62E27C4280DE1209FE80D6C0D0C0E03B
:20006000D2D3106E0DEAB50909C2A8D0E0D0D0C28922A80AE6F20ABA20027A10EAB509EBEB
:2000800080E7C0A8C2A8C0D0D2D3306E07313320B2FD115CC0E0E9B50A0B20B208D0E0F2DE
:2000A000D0D0D0A822D0E0F709B920027910E9B50A02D26ED0D0D0A8D2A822307A01223057
:2000C000E717B50712206F0DC0E0E50BB50C04D0E08004D0E0C322F5073133206FFD80230B
:2000E000307A012230E717B50712206F0DC0E0E50BB50C04D0E08004D0E0C322F507A26F70
:20010000500122C0A8C2ACC0D0D2D3C0E0EBB50C0F20680CD0E0F599D268D0D0C3D0A822FD
:20012000A80BD0E0F60BBB62027B42EBB50CEBD26F80E7758A00758C0022313320B3FDE208
:20014000227401F2752D02752E00752F00750910750A10750B42750C4275204B75210A7594
:2001600005007506037507007523FF7524FF7525FF7526FF7527FF752801752980783076A9
:200180000008B842FA758161758921758DFF75884075B8027964313AB4000CD9F9D2D5758A
:2001A00022037506014189B401EC313AB403004002D275313AF5223075024189D2AF900183
:2001C000C875F00C7172800C060033060035060036060037313AB406FB313A54C06004D2B5
:2001E00070422E313A313AF52A313A313A135005752B0C800B135005752BF48003752B0096
:20020000313A313A135005752C0C800B135005752CF48003752C0090027075F004717231C8
:200220003AB40CFB313A7A0B313AB44B471A313AB45941313A1392781392721392711392FB
:200240007413927313927A139269313AF505313AF506313AF528313AF529313AF526313A18
:20026000F527313AF525313AF523313AF52480060C1FC10C51EC74091182740B1182313A8E
:20028000B40BFB2027031219FE759870D2AFD2ACD2A9D28C519880FC3133207BFD30B31088
:2002A000307F03021237E53060EE207FEB020EC0E2FAFBB4680280074016B4F8005011E4C1
:2002C0007803D6F9B408004007C39408F9430308901BF17C2CEC1493B50307EC14239002E0
:2002E000F173DCF1EA901C1D93FA6004313ADAFC2261AC61C361C961CF61E161E961F061FD
:20030000F78107811581238134813D814B8171817F818D819B81A981CC81DA81E581F1A17E
:2003200010A113A11DA143A15BA177A186C1DDC1FAE11CE147E1566149614C614F6152614C
:20034000556158615B615E61610207660207740207830207A00207B40207FE020850020908
:20036000420209B2C2AC7B00EB9311820BDAF9D2AC22C000750000E5009311820500D5F0FC
:20038000F6D00022C000A805206909C0E0E928540FF8D0E048C0E07401206908A80108E437
:2003A000D333D8FD4237D0E0D00001BB20D5137409C2AC1182740B1182307904741511824C
:2003C000D2AC22753034021237753033021237C2AC74FD11827800E6118208B880F9D2AC1C
:2003E00022313AF8313A66F622313AF8313AF6227A0351ECFA41ECC2ACEA11829004037ACC
:200400000461660000000020D50122D26C9004147A0161641420D50122C26C9004227A0148
:2004200061641574E3522D9004317A037164021B24080A1490043B7A02616412FF7A0251A0
:20044000EC9004487A0361640D0000313AF8313AF9313AFA740CC2AC1182EA1182B81F097B
:20046000B9F206740111828003E41182DAFBD2AC2220D50122D26A90047E7A0161640B2083
:20048000D50122C26A90048C7A0161640A20D50122D26B90049A7A0161640920D50122C228
:2004A0006B9004A87A01616408313AF8313AB43310B8000DEE131350082069059004CA80EB
:2004C000039004C87A026164060006C1313AFA51EC9004D87A02616405FF9004E17A046108
:2004E00064040200FF313AC2ACE50211827A3B816990136578007906E89311BB08D9F93150
:200500003A11BB793B313A12136BD9F974F701BB02137990051A7A036164010103C2ACEA51
:200520001182EA540FC39407F8E50613D8FD7401400274FF118290053D7A066166000000DC
:2005400000FF00313AB48003021A6AC0E074807184D0E0243C11BB747F01BB74C0450511D1
:20056000BBE411BB20690F30700C790174C07507007184E401BB22BAC902C27030D5062009
:200580006903021A6A22313AFC7A0551ECFB313A30D510201F0D74B07184E52311BBEBC3C2
:2005A0001311BB20752DB90108D270A269B0D54022B9000FE522B403005008BC2E00400399
:2005C000BC326E30730A74C07507007184EC11BBE960012220D5FC9006257A0C7164313AD7
:2005E000B4063E313A54C0532E3F422E313A313AF52A313A313A135005752B0C800B135087
:2006000005752BF48003752B00313A313A135005752C0C800B135005752CF48003752C0087
:200620002251B180B90600330600350600360600377A0C1219EADAFB9006D37A0471643113
:200640003AB40C028005FA51E480F4313A7A3BC2AC120A4574031182E41182313A1182DA2E
:20066000FA7413118274091182740B1182D2AC7A0C1219EADAFB9006D77A067164313AB475
:200680000D4C313AFB313AFAC2AC740F1182741F118274F21182EB1182EA1182740F118282
:2006A000E4118274281182EB75F00A84901DE86001931182E5F0934A1182D2ACBC2E0302E8
:2006C0001379BC2F0261C3BC300261C9A15BFA51E480AA0C01403B1100FF0D005A201F18BA
:2006E00030690620D503BA780F74B07184E52311BB313A03C2E701BB213A207404313A21E3
:200700003A313A901D1D9330E702213AC0E074B07184D0E011BB313A244001BB3027022129
:200720003A790074B07184E52411BB313AC313FB11BBA269B38270400122790174B071846A
:20074000E52411BBEB01BB302F012274B07184E52511BBE401BB302F012274B07184E52567
:2007600011BB747F01BB74B07507007184744011BBE401BB74B07507007184744011BB74C0
:200780007F01BB303F05303811213A74B07184E52711BB313A03C2E701BB74D0718480F366
:2007A000303702213A74B07184E52611BB313A03C2E701BB304F0530482A213A313A600D59
:2007C000A272B0E74007A2E7B072400122C0E074B07184E52911BBD0E030E706F414B4807D
:2007E000011401BB74E07184E411BB313A207206B4800104F404032440C2E70200BB3047B7
:200800000630402F02013A12013A600DA271B0E74007A2E7B071400122C0E074B0120384E1
:20082000E5281200BBD0E030E706F404B48001140200BB74E0120384E41200BB12013A2008
:200840007106B4800104F404032440C2E70200BBD279B90200500330781574A0120384124E
:20086000013A243C1200BB12013AD3330200BB12013A12013AD333206966B90163AA34C3B3
:200880009A605C8532F020E73784C5F023B5F000400205F0C5F0253430E702747FF5346042
:2008A00013C39536B40B004036B4F6005031253630E701E4F53674D0120384E5360200BB00
:2008C000F40484C5F023B5F000400205F0C5F0FAE534C39A20E705B40B0050C1E480BE22A3
:2008E000AA33C39A60F98531F020E73784C5F023B5F000400205F0C5F0253330E702747F30
:20090000F5336013C39535B40B0040D3B4F60050CE253530E701E4F53574D0120384E5359E
:200920000200BBF40484C5F023B5F000400205F0C5F0FAE533C39A20E705B40B0050C1E4E6
:2009400080BE748012038412013A243C30D521C0E0C3941020E71775F00884B40A00500EC7
:200960002438F874FF05F0C333D5F0FC56F6D0E01200BB12013AD333D3331200BB20691B71
:20098000B90116D5322B753400E536602475360074D0120384E40200BB5016D531137533BD
:2009A00000E535600C75350074D0120384E40200BB22749012038412013A243C30D520C038
:2009C000E0C3941020E71675F00884B40A00500D2438F8E405F0D333D5F0FC46F6D0E012B5
:2009E00000BB12013AD333D3331200BB12013A206909B90104053280045002053122E59996
:200A0000307A07C0E01200FED0E020E705C020C02122B4F0004007540F23900A4C737E008E
:200A2000780ED6C2E7C423FD206915EEC39505540FB40800500FF808FEE50613D8FD500540
:200A4000900A8FED7375204B75210A22416C220041454145220022002200220022002200C4
:200A600022002200220022002200416F0210E620D51774131200827409120082740B12005B
:200A8000823079057415120082750700020A4541A0612761C58113C183419DE1EC02107E9A
:200AA000A2D5B06A5003020A457520B075210A22C3943CFF7520BB75210A220313541F507D
:200AC0000820D5050430E50114FDA269B0D5401374D82069012E120082EF120082ED1200EC
:200AE0008241A930701A74C0552EB44009EFC3952A20E70C8020B48007EFC3952A20E7162F
:200B000074D8120082EF252B120082ED12008274C0552EB4C09374D9120082EF252C1200B0
:200B200082ED1200828082A2D5B06A5003020A4575203775210B22C3943CFF7520427521ED
:200B40000B2270077D10120ACA80E50313541F500820D5050430E50114FDA269B0D540182B
:200B600074D02069012E120082EF120082ED120082E4120082020B3030701A74C0552EB407
:200B80004009EFC3952A20E70C8024B48007EFC3952A20E71A74D0120082EF252B1200826C
:200BA000ED120082E412008274C0552EB4C08174D1120082EF252C120082ED120082E4126C
:200BC0000082020B30E522B403005003020A45A2D5B06C40F77520DC75210B22C3943CFF64
:200BE0007520E775210B2203543FFD74682069012E120082EF120082ED120082A2698270FA
:200C0000B0D550D17469120082EF120082ED12008280C2A2D5B06A5003020A457520237515
:200C2000210C22B420005003020C79B44003020DFE500775201C75210C22B460005003027E
:200C40000DB2B473005003020D62B47A0040E420D5E1FF306906EEB505D97E0075206375B8
:200C6000210C22FDEFC3947A23900C6D73C13DC13FC141C14AC15EC15EB5282E75208375E8
:200C8000210C22207102F404FF74802069012E120082EF120082A2698270B0D550097481E8
:200CA000120082EF120082020C1CB5292E7520B475210C22207202F404FF74882069012E9B
:200CC000120082EF120082A2698270B0D550097489120082EF120082020C1CB5262A75204A
:200CE000E575210C2223FF74902069012E120082EF120082A269827082D550097491120092
:200D000082EF120082020C1CB5272A75201275210D2223FF74982069012E120082EF1200B7
:200D200082A269827082D550097499120082EF120082020C1CB5232D75203F75210D222375
:200D4000FF74782069012E120082EF120082A2698270B0D550097479120082EF12008202F8
:200D60000C1CC39440FF75206D75210D22307440C39440F5F0EF901D829320E733FD74E052
:200D80002069012E120082ED120082901DB5EF9330F71120E703E48014E5F0B4C000500D42
:200DA00074C08009C2E7B5F0004002E5F0120082811CFF7520BA75210D22302F03020C1C41
:200DC000FDE525B50FF7BD001974B82069012E120082A2698270B0D550E374B9120082028B
:200DE0000C1CBD7FD874B02069012E120082A2698270B0D550C774B1120082020C1C752036
:200E00000575210E22B4001974A82069012E120082A2698270B0D5502174A9120082020C20
:200E20001CB47F1674A02069012E120082A2698270B0D5500574A1120082020C1C811C8125
:200E40001CBD0004C269C165811CBD000F306902C165BE0007D269120A6FC165811CBD002F
:200E600002C165811C74F02E1200827480120082A2698270500A74F1120082748012008227
:200E8000020C1C207303020A45A2D5B06B5003020A4575209975210E22601AB4330050F274
:200EA0007830B600EDF5302069E8EEC31313134230926D80DD2069DA74C82E12008280D2E6
:200EC000A269B0D5402A74C05530A26D33333344C0C2AC120082743F553012008275300040
:200EE000C26D900EEA7A060203660000FFFFFF00C2AC7402120082E530120082D2AC1201A1
:200F00003AB4020280051202B180F3C2AC120A457403120082E412008212013AF8120082F7
:200F200074C058532E3F422EC2706002D27012013AF8120082E8790513D9FD5006752C0CF4
:200F400013800B135005752CF48003752C00135005752B0C800B135005752BF48003752B14
:200F600000781E12013A120082D8F812013AF52A120082781A12013A120082D8F87413124E
:200F800000827409120082740BF81200823079067415F8120082D2AC12013AB500028006E7
:200FA000FA1202E480F2C2AC900FE375F006120372E53075F00A84901DE8600193120082C6
:200FC000E5F093120082900FE975F003120372E530120082E41200827530007410120082C0
:200FE000D2AC221100FF0F00280F1FF2A2D5B06A5003020A457480B5280302103FB529F2C0
:201000007520077521102275200E75211022FF74882069012E120082EFC333C3948020726C
:2010200006F404B4800114FF120082A2698270B0D550CD7489120082EF120082021000759C
:2010400020467521102275204D75211022FF74802069012E120082EFC333C3948020710626
:20106000F404B4800114FF120082A2698270B0D550CD7481120082EF12008202103FA2D529
:20108000B06A5003020A4575208E7521102223FD74982069012E120082ED120082A2698221
:2010A00070B0D550E27499120082ED12008280D7120133D021D02022D00DD00E11B075F066
:2010C000F052F0C5F0701AC5F0C4FF11B075F0F052F0C5F0700BC5F0780FD6EFC00EC00D03
:2010E00022410C020A4520D5FA2075F711B3B408F211B370EE11B3B44BE911B3B459E411AF
:20110000B0701011B0B4350040024114F530D27F020A45D27B11B0B43402800221B511B086
:2011200013927813927213927113927413927313927A13926911B8B411004002410CF505F0
:2011400011B8F50611B8317CF52811B8317CF52911B83190F52611B83190F52711B831A0BF
:20116000F52511B83190F52311B83190F5242027031219FE121B35C27B020A45B420005089
:201180000122B4800122B4FF0122D0E0D0E0410CB42000500122B4FF0122D0E0D0E0410C88
:2011A000B44000400AB46000500122B4FF0122D0E0D0E0410C40024114B4332E7D0112109B
:2011C000B0B50DF3FF7403120082EF1200827E3B1210B0C4FF1210B0780FD6EF120082DE3F
:2011E000EF0DBD33D9C27B020A45FF7403120082EF1200827D3B1210B0C4FF1210B0780F69
:20120000D6EF120082DDEFC27B020A457D3CE4120082DDFA75F010901222120372C27B0214
:201220000A45101100FF0E0020083D67004F05051D050F006AC100C29CA27AC0D0C27A1258
:201240000A457507009012327A051203647408120082740A120082E522B40300400D741442
:2012600012008212013AB4140A801212013AB40A07800A1202B180EB1202B180EE7900129F
:201280001A6A2069083070057901121A6A78141219EAD8FB90136578007906E8931200BBC9
:2012A00008D9F8E5301200BBC27FE530753000B4343FE4A26933A27A33A27333A27433A2AD
:2012C0007133A27233A278331200BBE505716BE506716BE528716BE529716BE526716BE5DD
:2012E00027716BE525716BE523716BE524716B6141B4332A7B017402120082EB1200821272
:20130000013AB40213EB1200BB7C3B12013A716BDCF90BBB33E06141FA1202E480E1C0E0EE
:201320007402120082D0E012008212013AB4020B7C3B12013A716BDCF96141FA1202E48088
:20134000E974F71200BB7409120082740B12008230790574151200822027031219FED0D06A
:20136000927AD29C22F008004B597FC4FAE47802D61200BBEAC40200BB3075052230D501BA
:2013800022C29C120A457507007900121A6A20690730700409121A6A79019014057A271238
:2013A000036412013AB40C3912013A7A0512013AC0E0DAF97A031202ECC0E07A031202EC5A
:2013C000C0E012013AC0E07A031202ECFC901461E522B4030390142C7A35120364D27CA15A
:2013E00086FA1202E480BB12013320B3FAE2B4C0028196B4FC0302185DB4F80302170FFABD
:201400001202E480E20A0C0025050C0036010C1FF2020C002D011100FF0E017B0A6730005B
:20142000000000000067050E1FF601060E02002CC60A8E017B108E0020A680A7A05A26F95C
:201440008E0001BF0035F6002DF10185260139F7018586FCBDCD901F987ECD900F006A02E9
:20146000000E0CC02CC60A8E017B108E0020A680A7A05A26F98E0001BF0035F6002DF10150
:2014800085260139F7018586FCBDCD8A1F987ECD8A0F006A0CC012013AC0E07A061202EC16
:2014A000D0E0B41100C0E05028F9740F1200827401120082747C120082E975F00A84901D79
:2014C000E8600493120082E5F093120082E41200827A0C1219EADAFB901562E522B40303ED
:2014E00090155E7A0412036412013AB40C028006FA1202E480F212013A7A3B7403120082EC
:20150000E412008212013A120082DAF8741312008274091200827A0C1219EADAFB740F126F
:201520000082741F12008274F2120082D003D002D0E0C0E0C002120082EA12008212013AF2
:20154000B40915EBB411004008B42E02E10F0213E7E9142390156673FA1202E480DF0C02F4
:20156000413B0C01403BA186A18CA190A198A19CA1A9A1ADA1C2A1CDA1D1A1D5A1E2A1E611
:20158000A1F7C104C112E505F804C128A269C11DA27A4002C1BBC1D0A273C11DE50678079B
:2015A000334002D8FBE8021628A274C11DA828B8FF0308C191B8800578010216A6E8080877
:2015C000C128A271E433F86002C167C17CA82980DEA27280EFA826B8FF047800C191E80844
:2015E000C128A82780F1E525B4FF047800C191C3943FF8243FC128A823B8FF047800C1910D
:20160000E808C128A824B8FF057800021691E808C128A278E433F86002C1E5C1FAE433F874
:201620006003021652021691C0E090164A7A08120364D0E075F00A84901DE860019312006B
:2016400082E5F0931200820213E70F017F00000F018190165D7A0A1203640213E70F017F65
:2016600000000F01817E159016727A0A1203640213E70F017F673E0F01815B379016877A37
:201680000A1203640213E70F017F673E0F01810E0E90169C7A0A1203640213E70F017F0020
:2016A0007E0F018147479016B17A0A1203640213E70F017F670F0F01810D179016C67A0A93
:2016C0001203640213E70F017F007E0F01811C0F9016DB7A0A1203640213E70F017F0F179D
:2016E0000F0181051C9016F07A0A1203640213E70F017F00670F01811D309017057A0A1293
:2017000003640213E70F017F4E170F018115309017907A05120364C27CD0E0D0E0740E123B
:201720000082E412008274361200827401120082D0E0120082D0E0F8D0E0F9D0E0FAD0E079
:20174000FB740E120082E412008274251200827405120082D0E0120082EB120082EA120007
:2017600082E9120082E8120082121B35740B12008212013AB40B028006FA1202E480F23051
:20178000790574151200822027031219FED29C220F006AC100000000000000000000000071
:2017A000000000000000000000000000000000000000000000000000000000000000000029
:2017C000000000000000000000000000000000000000000000000000000000000000000009
:2017E0000000000000000000000000000000000000000000000000000000000000000000E9
:201800000000000000000000000000000000000000000000000000000000000000000000C8
:201820000000000000000000000000000000000000000000000000000000000000000000A8
:20184000000000000000000000000000000000000000000000000000000000000012013A3B
:20186000C0E0C39C30E702F404B403005005D0E00213E7D0E0FC901DF2E91493F5F0EC8470
:20188000B500030213E7F8E9142390188E7301B801C101CA01D801E101F101FA211E212C59
:2018A0002150215E2177219021AA21C321DCC0E07410120082D0E02211AE8805E804021669
:2018C0002811AEE813926902161D11AEE813927A40030216BB0216D011AEE813927302165B
:2018E0001D11AEAA000AE4D333DAFCF506E802162811AEE813927402161DB8220040030261
:2019000013E711AEB800067528FF021691B801067528800216A6E81414F52802162811AE45
:20192000E8139271400302167C021667B8220040030213E711AEB800067529FF021691B8BF
:2019400001067529800216A6E81414F52902162811AEE8139272400302167C021667E8B486
:20196000210040030213E711AE70067526FF02169114F526021628E8B4210040030213E724
:2019800011AE70067527FF02169114F527021628E8B4210040030213E711AE70067525FF94
:2019A000021691243FF525021628E8B4210040030213E711AE70067523FF02169114F52324
:2019C000021628E8B4210040030213E711AE70067524FF02169114F52402162811AEE8132E
:2019E000927840030216FA0216E5120133C0D0C000C2D378000000D8FCD000D0D022901AD8
:201A000040E522B40303901A1675F02AC0A8C2AC120372D0A8221100FF0E02001EB6002D5E
:201A20001F89B001852A02434C81022C0139F7018586FCBDCD901F987ECD900F006A0200FE
:201A40001100FF0E0CC01EB6002D1F89B001852A02434C81022C0139F7018586FCBDCD8A06
:201A60001F987ECD8A0F006A0CC0E537AA010A13DAFD40012230D5277A1078387B08E61395
:201A800040090ADBFA08B842F38014C0E07480120384EA1200BB74401200BBD0E080E374A9
:201AA000B0120384747B1200BBE41200BB74B012038474011200BBE41200BB74B012038403
:201AC00074401200BBE41200BB201F0F74B0120384E5231200BB747F1200BBB9000E30D568
:201AE00003753100753300753500800FB9010C30D50375320075340075360074D0120384B6
:201B0000E41200BB74E0120384E41200BB74401200BBE5377A087B001350010BDAFABB01DD
:201B2000028009227900516A09B908FA7837760008B842FA22C0A8C2AC901B9575F0071229
:201B40000372744B1200827459120082E4A26933A27A33A27333A27433A27133A27233A22B
:201B60007833120082E505120082E506120082E528120082E529120082E526120082E5273B
:201B8000120082E525120082E523120082E524120082D0A8221100FF0E1FC10CC2D3307BF6
:201BA0000412120C32758161307C0375816B74C0C0E0741BC0E074BFC0E0741BC0E03232EF
:201BC000C2AC120133120A4575070020D5197A3CE4120082DAFAD2ACD2AF207C05D29C0254
:201BE0000294C29C0213E7206A03306BE97A0880DF00F9FAFDFFFE0E70141513120D0C0B26
:201C00000A09080605040203F801E8F0FBC8C078E0FCB8B0A8A09890888068D8D0000001FC
:201C20003C0000020300000000030200040002000000000000000000000000000000000058
:201C4000000000000000000000000000000000000000000000000000000000000000000084
:201C6000000000000000000000000000000000000000000000000000000000000000000064
:201C8000000000000002020202020202020000000000000000010101010101010101010129
:201CA000010101010101010101010101010101010101010101010101010101010100000007
:201CC0000000000000000000000000000000000000000000000000000000000000070707EF
:201CE000070707070700000000000000000303030303030303020202020202020202020293
:201D00000202020202000000000000000001010101010101010000000001000000FFFFFFB3
:201D2000FF70FFFFFFFF08FF71FFFF60FF62FF64FFFF66FF68FF6A0AFF0CFF0EFF6CFF10CE
:201D4000FF12FF1416FF18FF1AFF6EFF1CFF1EFFFFFFFFFFFFFFFFFF09FF72FFFF61FF6342
:201D6000FF65FFFF67FF69FF6B0BFF0DFF0FFF6DFF11FF13FF1517FF19FF1BFF6FFF1DFF2F
:201D80001FFFFFFFFFFFFFFFFFFF093B1A4C1C4E1E502254245626582759295B2B5D2F6121
:201DA00031630E401042124415471749194B20522D5F040B3D00000000000000003F3F3F72
:201DC0003FBFBFBFBF3F3FBFBF07073F3FBFBFBFBF0F0F0F0F1F1F1F1F1F1F1F1F1F1F1FB3
:201DE0001FBFBFBFBF1F0F0F7E306D79335B5F707F7B108080802080078007800707070746
:201E000007800000000000000000000000000000000000000000000000000000000000003B
:201E20000000000000000000000000000000000000000000000000000000000000000000A2
:201E4000000000000000000000000000000000000000000000000000000000000000000082
:201E6000000000000000000000000000000000000000000000000000000000000000000062
:201E8000000000000000000000000000000000000000000000000000000000000000000042
:201EA000000000000000000000000000000000000000000000000000000000000000000022
:201EC000000000000000000000000000000000000000000000000000000000000000000002
:201EE0000000000000000000000000000000000000000000000000000000000000000000E2
:201F00000000000000000000000000000000000000000000000000000000000000000000C1
:201F20000000000000000000000000000000000000000000000000000000000000000000A1
:201F4000000000000000000000000000000000000000000000000000000000000000000081
:201F6000000000000000000000000000000000000000000000000000000000000000000061
:201F8000000000000000000000000000000000000000000000000000000000000000000041
:201FA000000000000000000000000000000000000000000000000000000000000000000021
:201FC000000000000000000000000000000000000000000000000000000000000000000001
:201FE0000000000000000000000000000000000000000000000000000000000000000000E1
:00000001FF
